:020000020000FC
:1000000052C109C009C009C009C0B7C0B7C0B8C053
:1000100029C148C1B4C01895189518950F92EF934F
:10002000FF932F933F931F931FB71F93209174004B
:100030002B50C9F4C79828E331E3E0918D00F0918B
:100040008E0088942E1B3F0BEAB5FBB5E20FF31F21
:10005000FBBDEABD10E418BFF0927400F0928D0071
:10006000F0928E0081C010917400E5E7F0E0E10F9E
:10007000FF0D0080E7E7F1E0202DE20FFF1DE20F0A
:10008000FF1DE20FFF1D2AB53BB52E0F3F1F3BBDE5
:100090002ABD20E428BF20918D0030918E002E0FC4
:1000A0003F1F20938D0030938E00E9E6F0E08894A6
:1000B000111F8894EE1FFF1FE10FFF1DC895E9E691
:1000C000F0E0E00DFF1D1091740013951093740083
:1000D00009940B00100016001C00220028002E00BE
:1000E00034003A00400046001091A10010FD929AA1
:1000F0003BC092981091A10011FD939A35C093983E
:100100001091A10012FD949A2FC094981091A10013
:1001100013FD959A29C095981091A10014FD969A07
:1001200023C096981091A10015FDC29A1DC0C298D7
:100130001091A10016FDC39A17C0C3981091A10099
:1001400017FDC49A11C0C4981091A00010FDC59A63
:100150000BC0C5981091A00011FDC69A05C0C698A5
:100160001091A00012FDC79A1F911FBF1F913F91D0
:100170002F91FF91EF910F9018951895189518955C
:100180002F933F930F92AF93BF93EF93FF931F92E1
:100190002F923F921F931FB71F9322E61BB114FBB0
:1001A00076F910FB2EF01CB1312E77FB36F011C022
:1001B0001CB1312E1AB111FB66F0109071001120A4
:1001C00009F442C010906E0020906F00121834F1B4
:1001D00032C010919F001F71232C269426942694E0
:1001E000211A31F0F0927100F0926E0078682CC004
:1001F0007068777F1AE0109372001FEF1093710000
:10020000F0926E0017E03122EBECF1E08894EE1FE3
:10021000FF1FE30DFF1DC89500926F0030916E0027
:10022000230FBB27A22F3C92339530936E001AE028
:100230001093720009C030916E00230FBB27A22FCC
:100240003C921FEF109370001F911FBF1F913F90B2
:100250002F901F90FF91EF91BF91AF910F903F9121
:100260002F911895AF93BF931F931FB71F931091B2
:100270006D00139510936D00155041F0A8E6109194
:100280006D00A10FBB271C911CB906C0539855984F
:10029000F0926A00F0926B001F911FBF1F91BF91F7
:1002A000AF91189518951FED1DBFFF24A0E6B0E093
:1002B000FD9219ED1A1BE1F71FE015BF10E01BBFFF
:1002C00010E419BF12E013BF10E01FBD12E01EBD05
:1002D000A89518E011BD112718BB12BB1CEF17BB66
:1002E0001DE711BB14E91AB91CE019B913E018B9DC
:1002F0002BD0E3D019D13CD17894DD24F2BE8CE729
:1003000092B79817EAF31CE7810FE8E9F1E013E0F0
:10031000D122ED2C8894EE1C8894EE1FFF1FEE0D69
:10032000FF1DC895E8E9F1E0E00DFF1DD3940994A5
:100330000400060008000A0032D0E2CFBFD0E0CFB0
:10034000F4D0DECF16D1DCCF77276627FBBCFABC12
:1003500019B71F7B19BF20E13327AEE9B0E01CB30A
:1003600010FBEEF33EBB11E01CBB1DB31D93339598
:100370002A952223A1F716B310FB70F90EF05298BC
:1003800011FB2EF017E619B9F0929F000895109115
:100390009E0019B9089501020101010103021090A4
:1003A0007000112009F487C0F0927000E7EEF1E0D0
:1003B000109062008894111C8894EE1FFF1FE10DBD
:1003C000FF1DC895E7EEF1E0E00DFF1D0994080060
:1003D0001900230023002300230024004200F09290
:1003E000740010916300112309F406C0FBBCFABC31
:1003F00019B7106419BF5EC019B71F7B19BF5AC067
:1004000010916300E0E8F0E0E10FFF1D109164003F
:10041000108350C04FC01091630010FB56F0A0EA4B
:10042000B0E010916400A10FBF1D109165001C93F6
:1004300041C01CB311FBEEF3109164001EBB109180
:1004400065001DBBF89414E01CBB12E01CBB789443
:1004500031C01091630010FBFEF011FB66F0A0EAC2
:10046000B0E010916400A10FBF1DF0926A001C91D2
:1004700010936B001FC0A0EAB0E010916400A10FC0
:10048000BF1D1D912C913E91311B3323A1F7109379
:100490006A0020936B000EC01CB310FBEEF31091AA
:1004A00064001EBB11E01CBB2DB3F0926A002093C8
:1004B0006B0000C07460A8950895089577FB0EF056
:1004C00031C0579872FB2EF4737710919F0010681B
:1004D0000DC0209172002A952093720019F573FBCC
:1004E00077770EF41FC010919F001F7776FB16F9E7
:1004F00010936800F0927100F0926E001091680005
:1005000020916900120F20916A00120F20916B0058
:10051000120F10936C00F0926D0010916800539AC6
:100520001CB9559A579A0895089550907300552014
:1005300009F41DC0A7EBA65B50906300A51918F441
:10054000F092730014C0F0927300E6EBF2E050906A
:1005500063008894551C8894EE1FFF1FE50DFF1D56
:10056000C895E6EBF2E0E00DFF1D09940100089547
:10057000089510918C00112321F01A9510938C008E
:1005800038C0112710938B00E5E7F0E0E10FFF1D65
:1005900020813BE0E30FFF1D3081E3EAF0E0E10F53
:1005A000FF1D4081442309F44395522F531BA1F0B2
:1005B00030F45095541B51F048F0240F08C0752EAC
:1005C000741A21F019F010F0241B01C0232FE5E765
:1005D000F0E0E10FFF1D208310918B005AE0511BCA
:1005E00021F0139510938B00CFCF1091A2001093A0
:0405F0008C000895DE
:00000001FF
